:01000000FF00
:10F200000075B0FF75D80FE5D85408602FC390F192
:10F21000FD74009394FF700EC390F1FC74009394FE
:10F22000FF700302010090F1FD740093F5F090F17E
:10F23000FC740093F58285F0837400737581D0129D
:10F24000F280C298D29990F1FB740093F5F0C394C8
:10F25000FF60277550FF7551FF85F052309803020B
:10F26000F306D550F730980302F306D551EE3098E7
:10F270000302F306D552E502F20D3098FD02F306C3
:10F2800075985A75CBFF75CAFA75C8347533002264
:10F290003099FDE534C299F5990022E542C412F295
:10F2A000B7E54212F2B7E543C412F2B7E54312F2F2
:10F2B000B7753468519022540FC0E0C3940A10D738
:10F2C000092441F5345190D0E022D0E02430F534C7
:10F2D000519022C0337533FAE58954F04401F58921
:10F2E000756100C28C758CB8758A02C28DD28C2073
:10F2F000980C308DFAD533EB756101D03322C2986A
:10F30000859941D0332200209805C29902F3BFC2EB
:10F3100098D299C3E599942A600302F3AD12F65D81
:10F320006035F5F0C39454701475343F12F2907543
:10F33000345412F290749312F29002F3BFE5F0C3CA
:10F340009453C375343F12F29075345312F2907493
:10F350009212F29002F3BF788086E0C39446603840
:10F3600086E0C39447700261D9788086E0C39457E1
:10F37000602986E0C39452602586E0C394456021ED
:10F3800086E0C39453601D86E0C3944C601986E008
:10F39000C39450601502F3AD02F3C402F45302F3B8
:10F3A000F702F4DA02F52602F61D02F58475343F01
:10F3B00012F29075344312F29075348212F290C2B8
:10F3C0009802F24675344612F29075345712F29054
:10F3D00075349D12F29002F3BF0886830886827509
:10F3E000344751907534005190753447519075A849
:10F3F0000074007302F3AD7881864408864590F16D
:10F40000FF740093C3540C940C7002812375342153
:10F4100012F29075345212F2907473F53412F29025
:10F4200002F3BF854483854582C3E58394F230D7D8
:10F43000DCC3740093F54675345212F290C37452D3
:10F440002546F5F085463412F29085F03412F2909C
:10F4500002F3BF7881864408864508864690F1FF0E
:10F460007400935403C39403601675345712F290DA
:10F4700075345212F29024A9F53412F29002F3BFBF
:10F48000C3E54494F230D7E2C375F65575F6AA7514
:10F49000F65575BF048544F48545F58546F675F740
:10F4A00080854483854582740093C39546701575A5
:10F4B000345712F29075340012F29075345712F2EC
:10F4C0009002F3BF75345712F29075342112F29006
:10F4D0002478F53412F29002F3BF75F65575F6AA4A
:10F4E00075F65575BF0475F783900000C3740093DB
:10F4F00094FF701DA3C3E58394F070F0753445123A
:10F50000F29075340012F29075344512F29002F3C5
:10F51000BF75344512F29075342112F2907534455E
:10F5200012F29002F3BF78818644C3E54494F1302F
:10F53000D70EC390F1FF740093C35430943060161B
:10F5400075345312F29075345212F29074A5F5345A
:10F5500012F29002F3BF75F65575F6AA75F6557559
:10F56000BF048544F475F50075F78275345312F2C3
:10F570009075340012F2907453F53412F29002F345
:10F58000BF02F60879807881864408864508866A35
:10F5900090F1FF740093C3540394036018753450C2
:10F5A00012F29075345212F29074502452F53412C3
:10F5B000F29002F3BF08C3E54494F230D7DFC3757D
:10F5C000F65575F6AA75F65575BF048544F485455C
:10F5D000F586468546F675F78085448385458274B1
:10F5E0000093C395467021080545E5457002054422
:0FF5F000D56AC375345012F29075340012F29040
:10F5FF0075345012F29002F3BF75345012F29075B9
:10F60F00342112F29075347112F29002F3BF75F635
:10F61F005575F6AA75F65575BF040000000075F70D
:10F62F008175344C12F29075340012F29075344C8F
:10F63F0012F29002F3BF75344C12F290753400122F
:10F64F00F29075346D12F29002F3BF74542275610B
:10F65F000051D38561E070F385413785413B753AA1
:10F66F002A7880E53A2541F53A51D38561E070DB80
:10F67F00A64108C3E894CF60D2C3D537E6883C18BB
:10F68F00883D18883E18883FA83DE6C3953A600329
:06F69F00745322740022E6
:10FA0000C0E0C083C082C0D0C0BF90F1FF7400933B
:10FA100054039403600D7CF0D0BFD0D0D082D0834B
:10FA2000D0E022C3EF94F010D70D7C0FD0BFD0D020
:10FA3000D082D083D0E022EFC3944030D70EC37C75
:10FA40000FD0BFD0D0D082D083D0E02275F65575CC
:10FA5000F6AA75F65575BF048FF48EF58DF675F719
:10FA6000808F838E82740093FDC39D700D7C00D0C7
:10FA7000BFD0D0D082D083D0E0227CFFD0BFD0D006
:07FA8000D082D083D0E02208
:10FB0000C0E0C083C082C0D0C020C0BF90F1FF74ED
:10FB10000093543003030303C2D79403600F7CF0B7
:10FB2000D0BFD020D0D0D082D083D0E022EFC394F9
:10FB3000EF10D70F7C0FD0BFD020D0D0D082D08391
:10FB4000D0E022EFC3944030D710C37C0FD0BFD099
:10FB500020D0D0D082D083D0E02275F65575F6AA99
:10FB600075F65575BF048FF475F50075F7828F2013
:10FB7000052005208F83758200740093C394FF7065
:10FB800017A3C3E583952070F07C00D0BFD020D0B0
:10FB9000D0D082D083D0E0227CFFD0BFD020D0D084
:07FBA000D082D083D0E022E7
:00000001FF
